:0200000001DF1E
:20002300309836C0E0C0D0C298A79930080AB74107200A16D20A8931300A07B70D04C20A09
:20004300D20909430180EAB5010B7401719790045B714280FED0D0D0E032EAB50101223038
:2000630099FDC2998A008699C208B60D02D2080A43028022200901220531433180C031A87A
:2000830031E6C394304050F5F09402504A752C04D031C0310531433180A831E6C3943040D3
:2000A30036940A5032D52CECD03185F030752C040531433180A831E6C39430C0E0E5307515
:2000C300F004A4252C2431F8D0E0F6D52CE231DE513D516EC20922D031C20922758E0175AE
:2000E3008152758780758922E5B0C4540790049893F58DF58BD28E7598527851760018B84B
:2001030001FAD2087A80798071A571DF740E7197748071977530021530513D516EE530706A
:20012300F675A890710974232530F8A62220020CE530B401037530FF053031BD20061431C6
:20014300C5B4090B76000522E522B404EF800204F631BD20071731C5600414F6800D7609AC
:200163000522E522B404EC512A800031BD20040B31C5B409047600803904F620050E31C589
:200183007006E522602C740A14F6702620000AE522B403037522FF0522200109E5227003E9
:2001A300752204152220030A31D27404760018D5E0FA31DE513D516E212774232530F88677
:2001C3002222E53075F004A424322522F8E622E53075F004A424322403F822752C04E530A6
:2001E30075F004A4252C90046F93C0E0E53075F004A4252C2431F886F0D0E0B5F003D52CD9
:20020300DD400122752C04E53075F004A4252C90046F93C0E0E53075F004A4252C2431F88D
:20022300D0E0F6D52CE122E53075F004A42432F8752C04760008D52CFA22E53090046893BD
:20024300C0E0719731D25164742C7178516451645164900464E52293F5F0D0E025F071974F
:2002630022E6516918222430717822752F04E53075F004A4252F2431F8E6C0E0742A252F3D
:20028300F8D0E0F6D52FE7E52C75F00AA4252BF52BE52E75F00AA4252D75F064A4252BF514
:2002A3002BE435F0F52CE52CC47E043392B351E4C2B251E4D2B251E4DEF1E52B7E08339256
:2002C300B351E4C2B251E4D2B251E4DEF1900490E53093F59051E47590FF51E4D2B351E489
:2002E300227F19DFFE22115D1177E580B4FFF774327F08C0E0115D1177DFFAD0E0D5E0F14B
:20030300E580B4FFE12251E9E580B4FF06115D117780F5F52022B40A0040022407243071D5
:200323007822C0E054F0C47119D0E0540F71192275F00A8424307178E5F02430717822E4E7
:200343009360057178A380F722F52B9360077178E52BA380F42274C0719722740171972234
:2003630043A0F0D2A1C2A0D2A2E5A0C2A2D2A2C2A220E7EC22D2A0C0E07186D0E0C4718614
:20038300716322C2A154F053A00F42A0D2A2C2A253A00F22C2A0C0E07186D0E0C471867108
:2003A300632253A00FC2A1C2A0C2A2749671CF71D771D771D77420718671637428719774F1
:2003C3000C71977406719774017197227F62DFFED5E0F92274307186743261CF8580203091
:2003E3000201229004A0714271599004AB714274077133710912035E9004B57142715990D0
:2004030004C27142710912035E9004D171427159900FF9E4937125900FF8E49371257109CE
:2004230012035E9004E07142900FFA914271599004E77142900FFD9142710912035E22E459
:20044300937133742D120378A3E4937133742D120378A3E4937133224F766572666C6F7714
:20046300000403020080C086C68CCC92D205090004050900040509000405090004050900D2
:2004830004050900040509000405090004FEFDFBF7EFDFBF7FFFFEFDFAF4E8D0A07543200E
:2004A300436F6E74726F6C0056657273696F6E3A2000436F70797269676874206279004D17
:2004C300617274696E20436C617573656E0053657269616C206E756D6265723A00446174B4
:0B04E300653A200054696D653A200066
:080FF8000000000000000000F1
:00000001FF
